:020000020000FC
:100000006DCEBBC10000000020C000008DC000000C
:10001000000097C00000000000000000020304067A
:10002000080C10182030406080000406080C1018DE
:100030002030406080A0C0000003070F1F000D0D9E
:100040000403060D0503030202004FB662FD0CC057
:10005000552041F00994C52DC095089483FDC7959E
:10006000C4BD64604FBE1895C0916400089483FDC0
:10007000C795C4BD6B7FC0916400CF3F09F41DC01C
:1000800070FF19C082FD05C04FBEC098C198C298CC
:100090001895C098C198C29876FD0DC065FD0BC03B
:1000A000C9E0CA95F1F7C091B100C0FD939AC1FDB6
:1000B000949AC2FD959A4FBE189524BCCC27C06473
:1000C000C8BF6460F8CFC7CF70FFC5CF65FDC3CF91
:1000D000C09AC1CF70FFBFCF65FDBDCFC19ABBCF66
:1000E00070FFB9CF65FDB7CFC29AB5CF939870FFB7
:1000F000B2CF65FDB0CFC7E0CA95F1F7C09AABCFDC
:10010000949870FFA8CF65FDA6CFC7E0CA95F1F718
:10011000C19AA1CF959870FF9ECF65FD9CCFC7E097
:10012000CA95F1F7C29A97CF4FB6C9B7CF7EC9BF6C
:100130006E7FCCB5CE0DDDB5DF1DDBBDCABD4FBEBC
:1001400018953FB68F7EABB7A074A2118061A0E076
:10015000ABBFA9B7AE7FA9BF7894A0916800AA23CE
:1001600041F085FD2AC0A0916800AA95A09368007F
:1001700024C040E050E085FD14C0A0B396FDA095DA
:10018000A2FD4FEFA3E096FDA2E0A5BFAA27A064C1
:10019000AABF8D7FA0B396FDA095A2FD5FEF451786
:1001A00041F7A0E461FDA093680085FD03C0A0E4D1
:1001B000A093680040939600816085FD0EC0A091D9
:1001C0006900AA2331F0A0916900AA95A093690063
:1001D00004C08061AA27A064AABF80FF0AC0A091C2
:1001E00096004A2F61FF8E7F85FD01C000C04093BD
:1001F00061004091B400443009F004C0A091610056
:10020000A0936300A52DA03408F06860A091600061
:10021000A395A093600051F0F894A9B7A160A9BF7D
:1002200084FF02C0A0E4ABBF3FBE1895A09174004C
:10023000A395A093740042E050916800552329F0E3
:1002400085FF03C05A9550936800A0919600A13095
:1002500018F0209299000DC020929A002092A300DD
:10026000A0919900AF5FA093990018F0AFEFA09311
:100270009900B09061005091B400523049F466FF8B
:1002800091F0A2E3BA1678F0A0918600A0936100E5
:10029000533049F466FF39F0A2E3BA1620F0A0917A
:1002A000C000A0936100509162005B1521F010F036
:1002B0005A9501C05395509362004A95D1F65091DA
:1002C000A300539509F45A955093A300A091A4005C
:1002D000AA95A093A40009F046C0A1E0A093A400B1
:1002E00045E0A091A5005A17F0F1A091A6005A1779
:1002F00028F441E0A3E0A093A40007C0A091A700C8
:100300005A1718F441E04093A400D0909C00C0908C
:100310006300DC14A8F0A091B400A430D9F066FD0D
:100320000FC0C0929C00539511F0A091A500A0931E
:10033000A300A1E0A093A400ACE3A093620013C0CB
:10034000A0919C00A40F20F45FEF50939C0002C08A
:10035000A0939C00A0919C00AF3F29F4AFEFA09325
:100360009A00A093A300F894A9B7A160A9BF84FF45
:1003700002C0A0E4ABBF3FBE18953FB64CB55DB51B
:100380008F7EABB7A074A2118061A0E0ABBFA9B70C
:10039000AE7FA9BF789481FD23C0A2E096FDA3E0C3
:1003A000A5BF8260A0B396FDA095A2FF05C04093B3
:1003B0006500509366001CC1A3E096FDA2E0A5BFB6
:1003C000AA27A064AABF8D7F85FF01C004C140E0B9
:1003D000A0B396FDA095A2FDFEC040939600EDC08F
:1003E000A3E096FDA2E0A5BF8D7F61FF71C0A2E0F2
:1003F00096FDA3E0A5BFAA27A064AABF8260409390
:10040000910050939200A0908F004A19B0909000F4
:100410005B09BB24A22C4C38520518F4209295009D
:1004200049C0A091D400AA2359F1483C520528F4B0
:10043000A0E1BA2EAAE0AA2E23C04836A1E05A07AE
:1004400028F4A8E0BA2EAFE0AA2E1AC0403DA2E0E0
:100450005A0728F4A4E0BA2EAEE1AA2E11C0403A01
:10046000A5E05A0728F4A2E0BA2EACE3AA2E08C0F1
:100470004839A8E05A0720F4A1E0BA2EA8E7AA2E2E
:10048000C42EA0919300CA1AD52EA0919400DA0A26
:10049000DD202AF4AFEFC094D094CA1ADA0A209271
:1004A0009500A8E0A210A0E0CA14DA0618F4A1E0B2
:1004B000A093950040939300509394004091910035
:1004C0005091920040938F005093900042E075C08D
:1004D000A09165004A1BA09166005A0B94FD60C074
:1004E00093FD5EC092FD5AC086FF03C0D52EC42E78
:1004F0000CC05695479591FD51C05695479590FD76
:100500004DC0D52EC42ED694C79461FD19C0AC2D14
:10051000AC51AD2DA24008F005C0DD2089F4AC2D12
:10052000A85C70F4A0916700A395AA2311F0A09392
:100530006700AA3008F44FC02092960081604BC03B
:10054000A0916700AA2319F0AA95A0936700A22C96
:100550005091BA0097FD02C0A090C800AAEFAA0E61
:10056000A22DA21DCA18DA0A4FB74170442319F010
:1005700040E050E015C0AFEFCA16D20418F04FEFBC
:1005800050E00EC0A091AC00CA9E412D000C441F4B
:1005900050E008F012C04FEF50E00FC0569547955D
:1005A00094FF07C0552309F04FEFA42FA6954A0FDB
:1005B000521D4F3F520508F04FEF40939600816067
:1005C00061FF09C0AFE1A095A923AB299A2F8F7DC8
:1005D000BB2009F48062A0E4A093680085FF03C0FB
:1005E000AAE0A093680061FD03C085FD01C08F7E75
:1005F00085FD03C0A0E2A0936900F894A9B7A160AB
:10060000A9BF84FF02C0A0E4ABBF3FBE189511E0B4
:100610000AC013E008C01AE006C01EE104C014E6D8
:1006200002C018EC00C005E1BB27BA95F1F70A95A6
:10063000D9F71A95C1F708952AE338E709C020E3EE
:100640003CE806C02AE234EB03C025E238EC00C0E7
:1006500012E0BB279498BA95F1F7C19ABA95F1F7D1
:10066000C198BA95F1F7949ABA95F1F7123009F05A
:10067000C09A123009F4C29AB091AD00BA95F1F760
:10068000123009F0C098123009F4C298B7E8BA9550
:10069000F1F71A95F1F6022FB22FBA95F1F70A95F4
:1006A000D9F73A95A9F694980895221B39E0001FCE
:1006B0003A9509F40895221F211B18F4210F8894FC
:1006C000F6CF0894F4CF622C722CB0E08894B395E6
:1006D000221F331FE0F7379527958894912E802E9F
:1006E000020B130B10F4192D082D10F4889401C07F
:1006F0000894661C771CBA9571F7172D062D08957E
:10070000322D11232AF43A9500951095031B130BF3
:10071000F894029F712C002D129F912C802C7894BC
:10072000780C172D921C292DB4E06B2E2695179569
:1007300007956A94D9F7332321F000951095031B90
:10074000130B08950091B400043009F474C0B09103
:100750009600B95198F0B72FB67081F466FD2BC0A2
:1007600005E09090C600B92DBA9521F00AE0BA953F
:1007700009F002E1B0917B00B01BE0F066FF0AC017
:10078000B0919E00B0939C00BFEFB093A300B1E086
:10079000B093A400B0916100B093630020927E00FA
:1007A00020927F002092800020928100209282007F
:1007B0006F7B41C060649090C600B92DBA9579F402
:1007C000B0916200B095BB1FBB1F1B2FB7950B2FBD
:1007D000B12FB170B3951B2FB02FBE7F25C0B92D9F
:1007E000BA95BA9581F4B0916200B095BB1FBB1F5A
:1007F000BB1F1B2FB7950B2FB12FB370B3951B2FBA
:10080000B02FBC7F14C0B0916200B095BB1FBB1F5E
:10081000BB1FBB1F1B2FB7950B2FB12FB770B39505
:10082000B3951B2FB02FB87FB0540B2F1209009334
:100830007E0010937F00089510917B001695009123
:100840007A000795B0917E00B01B0B2FB0917F000E
:10085000B10B1B2F28F40038BFEF1B0740F009C075
:100860000F37120508F405C00FE710E002C000E8DA
:100870001FEF00938300109384000895009183007C
:10088000B09180000B0F10918400B09181001B1F6C
:1008900020E03091840033230AF42A95B09182003D
:1008A0002B1F1AF4203F40F00AC02F3008F407C075
:1008B0000FEF1FEF2FE003C000E010E020EF3091BA
:1008C0006300B0919B003B1718F4323030F009C040
:1008D000B0918400BB235AF004C0B0918400BB23C4
:1008E00032F40093800010938100209382000895D9
:1008F0002091D70000918300000F10918400111FF8
:10090000FFDE11232AF40038BFEF1B0740F009C0B7
:100910000F37120508F405C00FE710E002C000E829
:100920001FEF002352F0B0916200B01B0B2F18F0A4
:10093000013008F00AC001E008C000950F5FB091D7
:1009400062000B0F08F001C00FEF009385000895BF
:100950002091D8000091810010918200D1DE1123F6
:100960002AF40130BFEF1B0740F009C00F3F12050A
:1009700008F405C00FEF10E002C001E01FEF1123E3
:1009800052F0B0918500B01B0B2F18F0013008F029
:100990000AC001E008C000950F5FB09185000B0F01
:1009A00008F001C00FEF0093630008950FEF677F19
:1009B00071FD29C072FD09C06860B0917B00BA303A
:1009C00020F0B52DB03408F4677FB091D300BB237D
:1009D000D1F0B0917B00BB23B1F00FEF10917B0001
:1009E00064DEF894B091730072FDB5E00B9F112D99
:1009F000002D7894112309F00FEFB0919E000B1792
:100A000010F400919E0000939D00089500917A00DB
:100A100010917B0000541140B0919D0010F4BA95E4
:100A200001C0B39511F0B0939D000895EFD3B0E0ED
:100A300074FDB1E0B06CB7B9B6B1B068B064B6B926
:100A4000E6DDB0E074FDB1E0B06CB7B9B6B1B06846
:100A5000B064B6B9B6B1B6FDFDCF04B115B1B6B14B
:100A6000BF77B6B92AD42DE62093A800222309F433
:100A700041C030E03093A900732E7694622E6694C4
:100A8000620E731E262D372D0217130778F0809003
:100A9000A800BDE6B80DB093A8008090A900B0E012
:100AA000B81DB093A900260D371DEECF8090A80089
:100AB0009090A9001091A90016950091A8000795A3
:100AC0001695079523E0169507952A95E1F720914D
:100AD000B5002A9529F42092A8002092A9000AC006
:100AE0002A9521F0800E911E2A95E1F78092A800A8
:100AF0009092A90008952091B500B6B1B6FDFBCF44
:100B000004B115B1B6B1BF77B6B9B091AA00B3952B
:100B1000B093AA00B83060F12092AA00B091D20040
:100B2000BB2321F1112329F0B091AB00BF3F61F04D
:100B300009C0B091AB000B1739F020F4BB2321F0B2
:100B4000BA9502C0B395E1F300919B00B093AB005E
:100B5000BA3F50F400ECB93F38F400E8B83F20F455
:100B600000E4B73F08F400E000939B007F7E089507
:100B70002130B1F00F3FB3E01B0790F4BDE6BB237B
:100B800079F0B091A8000B17B091A9001B0740F4B1
:100B9000B0919B00BB2359F0BA95B0939B0007C05E
:100BA000B0919B00BF3F19F0B395B0939B000091AB
:100BB0009B00B0916300B01B10F400916300B091F2
:100BC0009C000B1750F000919C00B0919C00BF3F1F
:100BD00021F0B0919C00B0939B00502E00936400D4
:100BE000B091AA00B73009F47061089502E3F89457
:100BF000B091D9000B9F012D000C001F7894B0918B
:100C00009B000B1710F000919B0000936100009374
:100C10006300502E0093640000939E00089520927C
:100C20007A00B0EFB0937B000895F8940CB51DB531
:100C30002091740078943091750060907600009354
:100C4000750010937600031B160971FD03C077FD34
:100C50007DC027C07090770020937700270922235A
:100C600011F00FEF1FEF8090780090907900309393
:100C70007800609279000091750010917600081953
:100C8000190920917A0030917B0036952795020F43
:100C9000131F10F40FEF1FEF00937A0010937B00E7
:100CA00029C020917A0030917B003901B4E08B2E6D
:100CB000B2E09B2E343010F08A949A94383010F0C1
:100CC0008A949A94769467948A94E1F7261937095E
:100CD000992021F0169507959A94E1F7200F311F7E
:100CE00020937A0030937B0028F43FEF30937A0012
:100CF00030937B00323008F4706871FF02C0B3E0BB
:100D00000DC0B091C40000917100023838F0B39565
:100D1000003A08F0B395B63008F0B5E09B2EB4E089
:100D20008B2E10917B0000917A0024E01695079598
:100D30002A95E1F70819120928F0B02FB250B12F07
:100D4000B20910F402E010E0980126C020917A0068
:100D500030917B003901769467946694669466942A
:100D60002619320906950695200F321D20937A0028
:100D700030937B00323008F07F7704E0369527957A
:100D80003695279526952695201B10F0223008F4DD
:100D900022E089019090C40060FDFECFE0908B00BE
:100DA000F0908C006160B9B7B061B9BF380177FDD0
:100DB00041C07694679400938B0010938C00B92DFA
:100DC000B330E1F0B0FD04C0060D171D930106C05D
:100DD000000F111F0250120922E030E0B92DB3308C
:100DE00068F020938D0030938E000093870010935D
:100DF00088006092890070928A003AC000938D004A
:100E000010938E00209387003093880060928900B1
:100E100070928A0071FF0DC0BFE0B0938D002092E8
:100E20008E00B093890020928A00B0938B002092AC
:100E30008C001EC0669400938B00B92DB33091F0E6
:100E4000B0FD03C0060D262D03C0000F025022E0A6
:100E5000B92DB33038F020938D0000938700609255
:100E6000890006C000938D0020938700609289005E
:100E700000917C0002FD0350013031F495FD0FC05C
:100E8000B0B7B77FB0BF11C0023039F4B0B7B860A7
:100E9000B0BFB4E0B06CB7B908C095FDF1CFB0B742
:100EA000B860B0BFB5E0B06CB7B90091A200000F58
:100EB00010F4BBE60B270093A20060FDFECFB2E06A
:100EC000B0936E006160B9B7B061B9BFB72FB670AB
:100ED000D1F020917A0030917B0036952795369598
:100EE000279571FF02C0B0E43B0FF8940CB51DB517
:100EF000020F131F1BBD0ABD6160B0E1B8BFB9B7D7
:100F0000B061B9BF78940895606120927D0020E0BF
:100F100067FD20E206C0606120927D0020E267FD4F
:100F200020E001E011E077FD11C0B72FB67009F0A5
:100F30006F7E14E100917B00069509F403950F3054
:100F400008F00FE071FF02C004E114E160FD0FC082
:100F5000B0917D00BB2359F071FF06C0B0916E00C7
:100F6000BA95B0936E0011F4706249C0ABDFB0B7B0
:100F70003B2FB77FB0BFB8B1B0B733FDB860B0BFDB
:100F8000B0917D00B395B0937D00B8B177FD06C0F8
:100F9000B1E071FDB3E0BA95F1F7B8B1B072B21734
:100FA00009F022C071FF05C00395011708F00A95EA
:100FB000CDCF64FD05C00395011708F0B2CFC6CFB1
:100FC0006F7EF8943CB56DB470907A0080907B0091
:100FD000370D681C6BBC3ABD6160B0E1B8BFB9B7F2
:100FE000B061B9BF78949DCFB0916D00B13008F475
:100FF00098CF64FD96CF0A9509F0A8CF7F7D209108
:101000008D0030918E00F894B0E1B8BF0CB51DB5DD
:10101000020F131F1BBD0ABDE0908700F0908800EF
:101020006160B9B7B061B9BF7894B72FB67039F0C5
:10103000B0916D0072FFB395B0936D0009C075FF5C
:1010400007C067FD05C064FD03C0BF91BF91EDC43B
:10105000089500E063FF03C064FF01C001E0F8945D
:1010600010917100B7E01B9F212D102D7894200F57
:101070002695179526951795269517951093710027
:10108000183718F4B8E7B093710000917100B0916F
:1010900072000B1720F06062C098C198C29860FD82
:1010A000FECFE0908900F0908A006160B9B7B0612E
:1010B000B9BF0895B2E095FD0AC0F894B0937C00E2
:1010C0009498939A62FF01C0C29A7894F4C0F894FD
:1010D000B0937C009498959A62FF01C0C09A78946E
:1010E000EAC0B3E082FF24C095FD11C002E0F8948D
:1010F000B0937C00E0E8F0E00093B100C2989598CE
:1011000062FF02C0C19A01C0949A7894D4C002E0F0
:10111000F894B0937C00E0E8F0E00093B100C09850
:10112000939862FF02C0C19A01C0949A7894C3C098
:1011300095FD0BC0F894B0937C00EAE6F0E0C2980D
:1011400062FF01C0C19A7894B6C0F894B0937C0055
:10115000EAE6F0E0C09862FF01C0C19A7894ABC0A3
:10116000B4E095FD0AC0F894B0937C009398959AEA
:1011700062FF01C0C19A78949EC0F894B0937C003D
:101180009598939A62FF01C0C19A789494C0B5E093
:1011900082FF24C095FD11C001E0F894B0937C005B
:1011A000E6E7F0E00093B100C198949862FF02C0B6
:1011B000C09A01C0939A78947EC004E0F894B093EA
:1011C0007C00EAE8F0E00093B100C198949862FFD7
:1011D00002C0C29A01C0959A78946DC095FD0BC06B
:1011E000F894B0937C00E4E6F0E0C19862FF01C09F
:1011F000C09A789460C0F894B0937C00E0E7F0E087
:10120000C19862FF01C0C29A789455C0B6E095FDBE
:101210000AC0F894B0937C009598949A62FF01C03C
:10122000C09A789448C0F894B0937C009398949AAC
:1012300062FF01C0C29A78943EC0B1E082FF24C030
:1012400095FD11C004E0F894B0937C00EAE8F0E06A
:101250000093B100C098939862FF02C0C29A01C087
:10126000959A789428C001E0F894B0937C00E6E762
:10127000F0E00093B100C298959862FF02C0C09A56
:1012800001C0939A789417C095FD0BC0F894B09361
:101290007C00E0E7F0E0C09862FF01C0C29A789459
:1012A0000AC0F894B0937C00E4E6F0E0C29862FFD4
:1012B00001C0C09A78946F7D089523E630E0F9016B
:1012C0002092B100C098C198C2989398949895982C
:1012D0006B7F0895A2EBB0E007E00D9307E00D935C
:1012E00001E00D9304E00D930FEF0D930D9309E0D2
:1012F0000D9302E00D9301E00D9301E00D93AEEB31
:10130000B0E001E00D9300E00D9304EB0D930FEFBF
:101310000D930D930D9303E00D930FEF0D9301E0EB
:101320000D930FEF0D9305E20D9300ED0D9308E77C
:101330000D9308EC0D9304E00D930FEF0D9301E076
:101340000D9300E00D930AE70D930AE00D9300E082
:101350000D9301E00D9300E00D930FEF0D9300E06E
:101360000D9308952091B9008B7F233009F4846098
:10137000B091BA009F7DB1FD90629F7BB091BB00A0
:10138000B1FD9064223011F0886001C0877F08951C
:101390000A95E00FF21DB4910895ECE1F0E00091A0
:1013A000B200F6DFB093D700ECE1F0E00091B300BB
:1013B000EFDFB093D800EAE2F0E00091B800E8DF98
:1013C000B093D9000091D100002309F403950131B5
:1013D00008F001E1B02FB00FB00FB093A5001B2FA4
:1013E000B10FB10FB00FB093A600B10FB00FB00F97
:1013F000B093A7000091B800023008F402E0009317
:101400007300B091CE000FEFB23009F400EAB330B0
:1014100009F402E800937200E8E3F0E00091D500DF
:10142000B7DFB093A000089508952091C8003091CF
:10143000C900B091BA00B33009F43E5097FF02C022
:1014400020E03FEFB32FB21B6B2EB25810F4B2E87E
:101450006B2E00E00395609EB12DBD57D8F300932D
:10146000AC0008959068E1DFD8D820E030E0B0E12A
:101470006B2ECFD8B09196002B0F321D6A94C9F70E
:10148000B4E036952795BA95E1F7822E9F77CDDFA8
:101490000895F894E3E0F0E0B9E0B7BFB491B07814
:1014A000C1F3F894A895B1B5B861B1BDB0E0B1BDD4
:1014B000B4E0BEBFBFE5BDBF00DFB0E0B8BBB7E181
:1014C000B7BBB0E0B5BBB0E0B4BBB0E0B2BBB8E313
:1014D000B1BB2224A0E0B0E02D92AA31E9F7A0E64A
:1014E000B0E00FEF2D920A95E9F7B1E0B093A200BA
:1014F000F1DEDCD2B0E0B06CB7B9B6B1B460B068C0
:10150000B6B90091CA000093AD00B1E0B0936A0093
:10151000F89487D891D881D892D87FD893D87DD89D
:1015200054D37FD87ED87BD8F8940AEF1AEFA0B3B3
:1015300096FDA095A2FF1FC01A95C9F70A95B1F7AD
:10154000E0E0FCE1B591B43E39F4B591B03E21F450
:10155000B591BF3F09F40CC0E0E0F395F395B59168
:10156000B83F49F4B591B43931F4B591BA3A19F4A8
:10157000EE27F6950994F6DE10DF56DF56DF009170
:10158000CA000093AD0099DEB2E0B3BFB2E0BEBDC9
:10159000B2E0B5BDB1E5B8BFB9BFB0B70B2FB77FEB
:1015A000B0BFB8B1B0B703FDB860B0BF30D8789461
:1015B0003DDA20927000B3E096FDB2E0B5BFB0E432
:1015C000BBBFBB27B064BABF8D7F2BD8626033E04E
:1015D0002CE0B0919500BB2321F42CE03A9509F45E
:1015E000A3CF1BD880FFA0CF8E7FB0919600B230E2
:1015F00078F3B92FBF710091980000939700B093D2
:101600009800B01729F72A9521F76D7FB3E096FD72
:10161000B2E0B5BFBB27B064BABF8D7FB091D40034
:10162000BB2321F48062B92FB0709B2F8F7B209257
:101630006700F5D785FF05C0B0916700BA3008F0A4
:101640008064E7D702E085FF01C000E0B09196001A
:10165000B017B8F3F894F0D7EFD7EED77894E1D776
:1016600020928600D6D7B091BE00B13008F46EC08B
:10167000B0916A00B13008F469C085FD18C0B0911E
:101680009600BF3F08F462C0F894DFD77894C7D7BC
:10169000B0919600B130C0F7F894CED7BCD7CCD774
:1016A0007894BDD7B0919600BF3FB0F3C0C2B8E008
:1016B0009B2E9068F894B9DE7894B1D7F8949F7710
:1016C000B4DE80909600B0919600BF37789408F40D
:1016D00045C09DD7F894B9D778949A9451F7C2DE53
:1016E000B82DB550B093C9009CD7F8940CD272D2E3
:1016F0007894BAE09B2E9068F89497DE78948FD710
:10170000F8949F7792DE80909600B0919600BF3754
:10171000789478F77CD7F8948FD77DD78DD7789445
:101720009A9449F79FDEB82DBB5FB093C80079D774
:10173000F894E9D15ED2789472D7F89476DE7894F2
:10174000B0919600BF3F08F498CF71C20091960007
:10175000B09186000B1710F00093860060D701E06F
:10176000B091BA00B35009F405E0B0919600B017FB
:1017700008F078CFF89469D768D767D7789451D7AD
:1017800020926A0020926B0020926C00B0916B0056
:10179000B395B0936B00BF3F71F5B0916C00B395FA
:1017A000B0936C00B091CC0009E1BA9559F002E316
:1017B000BA9541F00DE7BA9529F00AEFBA9511F004
:1017C00020926C00B0916C00B017A8F076DD1FD7A6
:1017D000B0916C00BA95B0936C0020926B00B09100
:1017E000CB00B093AD00F89430D77894B091CA0094
:1017F000B093AD0014D70FD7B0916800BB2319F494
:1018000085FF01C091CE01E085FD01C006E0B091E9
:101810009600B01708F4BACF02D7B0916800BB2386
:1018200009F482CEF89449DD209261002092620092
:1018300020926300522C209264002092A1007894A0
:10184000B091B700BB0FB0939F0020927E00209212
:101850007F002092800020928100209282002092BE
:10186000AA0060E070E020927100B8E0B093AA0096
:101870007061CDD6B0E074FDB1E0B06CB7B9B6B16F
:10188000B068B064B6B9B6B1B6FDFDCF04B115B15C
:10189000B6B1BF77B6B9112309F00FEF0093AB00D3
:1018A0002AD9B8E0B093AA0070615CDDF894BFEF6C
:1018B000B0939B009BD9B0916100B0939B00B09313
:1018C0009C00B0939D007894B1E0B0936100B09318
:1018D00063005B2EB0936400B093A400B0919A00B3
:1018E000B093A300B091BA00B33019F49F7D87FD87
:1018F00090627160726020926D0088DC9EDC8FD9EE
:1019000094D98DD992D98BD906DB1CD7A2DBD2DB37
:101910008CD9FADA66FD90D777FF48D877FD76D86C
:1019200098DBDFDB82D9F7DA66FDA8D792DB18DC1B
:101930007CD9EADA66FDDCD78CDB29DC76D9EBDAF8
:1019400066FD06D886DB62DC70D9DEDAB0E074FDB5
:10195000B1E0B06CB7B9B6B1B068B064B6B979DB14
:101960006CDC63D9C8D871FF1EC0B0919E00B093E3
:101970009B00B0939C00B0919A00B093A300B1E09B
:10198000B093A40018E12CE0B0916D00B11728F0DD
:101990007D7F746020936F0006C0B0919600B130D7
:1019A00008F0B2CF4CC072FF11C067FD0FC0B091FC
:1019B0006F00BA9519F47B7F7860A6CFB0936F0063
:1019C000B0919600B13008F09FCF39C020927000DE
:1019D000B0919900B13058F0B0919E00B0939C0046
:1019E000B0919A00B093A300B1E0B093A400B0917D
:1019F00099000AEF1091D600112309F003E0B01707
:101A000008F01DC085FF04C0B0916800BB23B9F089
:101A100000EF67FF05C0B0919E00B0939B0000E20D
:101A2000B0917B00B01708F46FCFB0917000B39500
:101A3000B0937000B0919600BB2309F002C02092D1
:101A40007000F8943ADC8090B900B2E0B093B9002D
:101A500089DC8092B900209261002092620020927D
:101A60006300522C2092640020929F0060E070E09E
:101A70007894D5D522DC0091D600002319F0C09AC5
:101A8000C19AC29AB0E0B06CB7B9B6B1B460B068F0
:101A9000B6B985FF05C0B0916800BB2309F444CDF9
:101AA000B091BF00B13008F0CCCD6CCEEDE0F0E0ED
:101AB00023D0053A09F01BC0EEE0F0E01DD00A3556
:101AC00009F015C03AE0A2EBB0E0E3E0F0E014D09A
:101AD0000D9331963A95D9F739E1AEEBB0E0EFE0EE
:101AE000F0E00AD00D9331963A95D9F702C0F2DBB7
:101AF0000AD0E8E2F0E00895E199FECFEEBBFFBB2B
:101B0000E09A0DB308951ED03AE0A2EBB0E0E3E016
:101B1000F0E00D910FD031963A95D9F739E1AEEB5F
:101B2000B0E0EFE0F0E00D9105D031963A95D9F7AD
:101B300012D00895E199FECF0DBBEEBBFFBBE29A38
:101B4000E19A0895EDE0F0E00FEFF4DFEEE0F0E071
:101B50000FEFF0DF0895EDE0F0E005EAEBDFEEE0F7
:101B6000F0E00AE5E7DF08953091AE000091AF00A4
:101B7000313011F40093B200323011F40093B3000D
:101B8000333011F40093B400343011F40093C600E4
:101B9000353011F40093B500363011F40093B800DD
:101BA000373011F40093C400383011F40093B900B9
:101BB000393011F40093CE003A3011F40093BA009A
:101BC0003B3011F40093BB00089525E02AD52A95F7
:101BD000E9F7089531D533D535D537D51CD52CD572
:101BE0002ED530D532D517D527D529D52BD52DD5FE
:101BF00008952BD527D523D51FD50DD526D522D58C
:101C00001ED51AD508D521D51DD519D515D50895B8
:101C10008090AE009090AF000FD50ED50DD5FBD4BF
:101C20008A94D1F712D5F7D49A94E1F70895F894ED
:101C3000D1DF7894CADFC9DFB1E0B093AE00B1E084
:101C4000B093AF002092B000F894E2DF7894B5E052
:101C50006B2E70909600E5D4B09196007B16C9F774
:101C6000B13018F0BF3F40F107C07EDFF8944BDF82
:101C7000B1DFB8E0B1BDA9DF6A9459F7B091B00007
:101C8000B395B093B000B33008F4DECF9EDFB091CF
:101C9000AF00B395B093AF00F894B091AE00BA9591
:101CA000EEE3F0E0EB0FF21D049178940395B09110
:101CB000AF00B01708F4C6CF88DF87DFB091AE0061
:101CC000B395B093AE00B091AE00BC3008F4B7CF7E
:0E1CD00001DBF89418DFB8E0B1BD77DFDACBA6
:00000001FF
